:03000000022AD2FF
:0C2AD20078FFE4F6D8FD758142022B1954
:100E9E000A53746172743A20004950436F6E6E6546
:100EAE0063745245510A004950436F6E6E65637408
:100EBE00003E432C562C43432CC0E4E0EFF2E5F009
:100ECE0020D1E8EDEAEEEC49500A003E432C4D41AC
:100EDE00432C25303262583A25303262583A25304A
:100EEE003262583A25303262583A25303262583AD8
:100EFE0025303262582C4D414320E0E4F0E5F10AF2
:100F0E00003E432C5645522C20332E3120EEF2203B
:100F1E0025732025732CC2E5F0F1E8FF20495020FF
:100F2E00ECEEE4F3EBFF0A004E6F76203033203206
:100F3E003030370030383A35323A3031003E432CBB
:100F4E004C442C50524F473A202020202020202065
:100F5E002020202020202020202020202020202083
:100F6E002020202020202020202020202020202073
:100F7E002020202020202020202020202020202063
:100F8E00202020202020202020202020202CC4E0E3
:100F9E00F2E020EFF0EEF8E8E2EAE828F4E0E9EB20
:100FAE00290A003E2A2C312CCEF1EDEEE2EDFBE5C6
:100FBE0020EFE0F0E0ECE5F2F0FB20F1E5F2E5E207
:100FCE00EEE3EE20E8EDF2E5F0F4E5E9F1E00A00FB
:100FDE003E412C4130312C2562752E2562752E2511
:100FEE0062752E2562752C495020E0E4F0E5F12063
:100FFE00E0E4E0EFF2E5F0E00A003E412C41303251
:10100E002C2562752E2562752E2562752E2562752C
:10101E002C495020E0E4F0E5F120EEF1ED2E20F128
:10102E00E5F0E2E5F0E00A003E412C4130332C259C
:10103E0062752E2562752E2562752E2562752C49D8
:10104E005020E0E4F0E5F120F0E5E72E20F1E5F0A8
:10105E00E2E5F0E00A003E412C4130342C25627569
:10106E002E2562752E2562752E2562752CCCE0F12B
:10107E00EAE020F1E5F2E80A003E412C4130352C41
:10108E002562752E2562752E2562752E2562752CAC
:10109E00D8EBFEE70A003E532C4130362C25627504
:1010AE002CC2F0E5ECFF20EEE6E8E42E20EAE2E8C2
:1010BE00F2E0EDF6E8E820282A3130ECF1290A00BA
:1010CE003E2A2C312CC4EEEF2E20EFE0F0E0ECE5C2
:1010DE00F2F0FB20F1E5F2E5E2EEE3EE20E8EDF2D0
:1010EE00E5F0F4E5E9F1E00A003E422C5330312CF4
:1010FE002562752CC6E4E0F2FC20E7E0EFF0EEF19D
:10110E00E020F1EEE5E4E8EDE5EDE8FF20EEF2207B
:10111E00F1E5F0E2E5F0E00A003E422C5330322CCD
:10112E002562752CCEE1ECE5ED20F120F1E5F0E243
:10113E00E5F0EEEC20E1E5E720EAE2E8F2E0EDF69C
:10114E00E8E90A003E422C5330332C2562752CCF31
:10115E00E5F0E5E7E0EFF3F1EA20EFF0E820EFEE5F
:10116E00F2E5F0E520F1E2FFE7E820F120F1E5F00D
:10117E00E2E5F0EEEC0A003E422C5330342C2562B0
:10118E00752CCDE5F220EFE5F0E5E4E0F7E820E49C
:10119E00E8E0E3EDEEF1F2E8EAE820E220F1E5F036
:1011AE00E2E5F00A003E422C5330352C2562752CB8
:1011BE00CAE0EDE0EB20F8E8F0EEEAEEE2E5F8E06A
:1011CE00F2E5EBFCEDEEE3EE20EEE1ECE5EDE00A10
:1011DE00003E532C5330362C253032625825303297
:1011EE0062582530326258253032625825303262CC
:1011FE005825303262582C4D414320E0E4F0E5F1A1
:10120E0020F8E8F0EEEAEEE2E5F8E0F2E5EBFCEDD0
:10121E00EEE3EE20EEE1ECE5EDE00A003E454E4455
:10122E000A0044756D705820202020203030203068
:10123E0031203032203033203034203035203036DB
:10124E0020303720303820303920304120304220B5
:10125E0030432030442030452030460A003A2000EA
:10126E000A0044756D70442020202020303020303C
:10127E00312030322030332030342030352030369B
:10128E002030372030382030392030412030422075
:10129E0030432030442030452030460A00457272DB
:1012AE00206B657900526420656570726F6D0A005F
:1012BE005264204D454D0A00526420436F64650A06
:1012CE000044656275674950204F4E0A00446562BE
:1012DE0075674950204F46460A004465627567554A
:1012EE00736572204F6E0A004465627567557365AB
:1012FE0072204F46460A0044656275674D7367203B
:10130E004F6E0A0044656275674D7367204F4646FF
:10131E000A00436F6E666967206C6F636B210A006B
:10132E00577220656570726F6D0A00205361766585
:10133E0020656570726F6D210A00457272204D41F5
:10134E004321004C6F61643E3E002A003C41303127
:10135E003D003C4130323D003C4130333D003C418C
:10136E0030343D003C4130353D003C4130363D008F
:10137E004E4F4950004C494E4B434F4E5452005421
:10138E0052415353004652004E4F4C494E4B00496A
:10139E004E49004E4F4449414700003C21003C530A
:1013AE0030313D003C5330323D003C5330333D0034
:1013BE003C5330343D003C5330353D003C533036C9
:1013CE003D00FF137EFF1383FF138DFF1393FF1357
:0A13DE0096FF139DFF13A1FF13A853
:06331E000116000114007D
:10338900C2AFC28E438910758BFF758DB7D2ABD290
:043399008ED2AF22FF
:03001B00022A3680
:102A3600C0E0C083C082C0D0C2AFC28E758BFF75A6
:102A46008DB720060675A61E75A6E10514D202E509
:102A56001660020516E515D39401400215150519F1
:102A6600E519540F7050D20DE519543F701AD20073
:102A760090668DE0601204F0E0D394B4400A908032
:102A8600007480F0C2AF80FE906688E0600204F0B9
:102A9600906104E0600214F090668EE0D3940140E9
:102AA60003E014F03005020517E518D394644004DA
:102AB600D20680020518E513D3940140021513D2FD
:0C2AC6008ED2AFD0D0D082D083D0E032CE
:10088100C291C290D2B5C20A7D027C007F071233A9
:10089100018F24E524646060097D017F601232B913
:1008A100D20AE4FDFC7F0B1233018F24E52430E6EC
:1008B100097D04E4FF1232DDD20A7D017C007F074D
:1008C1001233018F24E5247008FD7FFF1232B9D263
:1008D1000A300A03126000C2AFC288C2A8C2AA7558
:1008E1008900122D67906341E0B4FA09A3E064CE58
:1008F1007003020981E4F52474392524F582E43476
:1009010063F583E4F00524E524B443EC906341747A
:10091100FAF0A374CEF0A374CCF0906347740AF09C
:10092100E4A3F0A304F0A3F090634C7403F0A37468
:10093100CCF090633D74FFF0A3F0A3F0E4A3F0903A
:1009410063587405F0E4F524E5242401FFE433FE43
:1009510074392524F582E43463F583E0FD123370A4
:100961000524E524C3944340DFE4F5A775A61E756D
:10097100A6E1907FF0F0A3F09080007480F080FEFB
:10098100D2AF90634C7403F0A374CCF0E490634B4A
:10099100F0122562EF60031219C7C2B51230E9C225
:1009A10006123090906358E0C3940350037403F02F
:1009B100D20AC20CC20BD293200A077E0E7F9E126E
:1009C1002648E4906578F0123389C2AFA37408F029
:1009D1009062B77424F0E4A3F0906341E09062B9AF
:1009E100F0906342E09062BAF0906343E09062BBA2
:1009F100F0906344E09062BCF0906345E09062BD8A
:100A0100F0906346E09062BEF0751501E490657A5E
:100A1100F0C207C208D2AF75A70775A61E75A6E179
:100A2100200A18AF24FE7D03122729E4FF12298C26
:100A31007E637F78E4FB7D0112280390668DE06080
:100A4100037401F0E4906104F0A37455F0A3748180
:100A5100F0E4F517E4F518906104E070031221EB5E
:100A610090668EE0B401119080007410F0E49066FD
:100A71008EF0D20AD20BD20C908008E0F52430E43B
:100A810005D2077410F0E52430E508D209908008FA
:100A91007420F0E52430E608D2089080087440F014
:100AA100E517D394034023908002E4F0908001F095
:100AB100908000F0E517D39406400FE4F517C203C8
:100AC10090657AF07515011230909080A0E0700366
:100AD100122EDC9080B8E07003122F569080D0E087
:100AE1007003122FD0908000E07013300710122491
:100AF1005E906334EFF0D39400400312002690809F
:100B010002E07006908000E06005D205020A55C23D
:100B110005E4F517906104E06003020A55300912FB
:100B2100122085906334EFF0D394004005E0FF126A
:100B310033AC200803020CB4121F10906334EFF0A1
:100B41007003020A55906378E054BF247F7003025A
:100B51000C17147003020BEF24026003020C4A20ED
:100B61000A077E0E7FA7122648300E792003769061
:100B71006350E07006906354E0605B906684E0FF30
:100B8100906350E0B50724906685E0FE906351E0E4
:100B9100B50618906686E0FE906352E0B5060C90AB
:100BA1006687E0FE906353E06E602B906354E06FC4
:100BB1007033906685E0FF906355E0B50727906636
:100BC10086E0FF906356E0B5071B906687E0FF90D3
:100BD1006357E0B5070F90657A7401F01233AD7574
:100BE1001501020CB490668474FFF0020CB4906697
:100BF1008DE060037401F090667CE0FF90637AE021
:100C01006F6003020CB490667CE004F0E4F515908B
:100C11006578F0020CB4300303020CB4906347E032
:100C21007003020A5512001ED203E4F5159065788F
:100C3100F090668804F0E490667BF0A3F0200A73DC
:100C41007E0E7FB5122648806A90668DE06003743F
:100C510001F0300352906378E020E74B90637AE033
:100C6100FF90667BE0FE6F600D906683E07007EE9B
:100C7100146F703F801390667BE004F0906334E062
:100C8100FFD3940440031233A89060007482F0A350
:100C91007401F090637AE0906002F07E607F007DE5
:100CA10003122E61020A55300E0920030690668454
:100CB10074FFF0200303020D69E515706B1231E139
:100CC100EF60207E647F78906479E02404FD122E29
:100CD10061906683E06003020A55906358E0F51560
:100CE100020A55906688E0D3943C403C906683E0CC
:100CF100703690668804F09062B6E0702B1228D7A7
:100D0100E4906478F0A37412F090667CE090647AC9
:100D1100F0A374FDF090610763A20190647C63A26B
:100D2100017F12121C95809B12339DEF601590601C
:100D3100007483F0E4A3F07E607F007D02122E61D7
:100D4100020A55E51564016003020A55906578E0D1
:100D510004F0E0C394055003020CC4C203E490659F
:100D61007AF01233AD020A55E51564016003020AF7
:100D71005590657AE014604024FE603C14700302D3
:100D81000E5124046003020A55E4F517200E139056
:100D9100657A7404F0906578E05401F075150102EC
:100DA1000A55E490657AF090657804F07515C8905D
:100DB100668474FFF0020A55906684E07003020EA7
:100DC100409064787480F090647A7401F0E4A3F048
:100DD100A304F0A37430F0A3747BF0E4F524747FD2
:100DE1002524F582E43464F583747DF07480252430
:100DF100F582E43464F583E4F0E524240790647912
:100E0100F07C667D8490634CE0FAA3E0FB7F0212E4
:100E11002BE37E647F78E5242409FD122E61906620
:100E210083E0601B12001ED203E4F515906578F093
:100E310090668804F0E490667BF0A3F0020A559076
:100E4100657A7404F0906358E02432F515020A556E
:100E51009080027410F0751503906578E06401FFCD
:100E6100F090657A7401F0EF7019906354E06013AB
:100E7100FCA3E0FDA3E0FEA3E0FF906684121889C5
:100E8100020A55906350E0FCA3E0FDA3E0FEA3E05D
:0C0E9100FF906684121889020A5580FE4A
:010E9D002232
:10002600906379E0B444047F0180027F0090637896
:10003600E0B447047E0180027E00EE5F604A906372
:1000460041E090637AF0906342E090637BF09063C6
:1000560043E090637CF0906344E090637DF09063AE
:1000660045E090637EF0906346E090637FF0906396
:10007600797452F09062B063A2019080A863A201E5
:100086007F06121C95020877906334E0C3940850EB
:1000960003020880906341E0FF90637AE06F60039B
:1000A600020880906342E0FF90637BE06F6003028A
:1000B6000880906343E0FF90637CE06F6003020872
:1000C60080906344E0FF90637DE06F6003020880E8
:1000D600906345E0FF90637EE06F600302088090C6
:1000E6006346E0FF90637FE06F60030208809063E1
:1000F60079E0B444159062B0E0B4FF0E63A20190BB
:1001060080A863A2017F06121C9590668DE06003AD
:100116007401F090668E7464F09063797452F09076
:100126006378E0646D60030202A37BFF7A0E79BFF9
:1001360012144A7BFF7A0E79D9906341E0F52DA31C
:10014600E0F52EA3E0F52FA3E0F530A3E0F531A30B
:10015600E0F53212144A752DFF752E0F752F367580
:1001660030FF75310F7532427BFF7A0F790F12140B
:100176004A7BFF7A0F794B12144A7BFF7A0F79B1CB
:1001860012144A7BFF7A0F79DE906347E0F52DA3C0
:10019600E0F52EA3E0F52FA3E0F53012144A7BFF1D
:1001A6007A107908906350E0F52DA3E0F52EA3E0D0
:1001B600F52FA3E0F53012144A7BFF7A10793690BA
:1001C6006354E0F52DA3E0F52EA3E0F52FA3E0F5AB
:1001D6003012144A7BFF7A10796490633DE0F52D66
:1001E600A3E0F52EA3E0F52FA3E0F53012144A7B29
:1001F600FF7A107987906339E0F52DA3E0F52EA3F9
:10020600E0F52FA3E0F53012144A7BFF7A1079A4AB
:10021600906358E0F52D12144A7BFF7A1079CE12BE
:10022600144A7BFF7A1079F7A20EE433F52D1214E7
:100236004A7BFF7A117927906683E0F52D12144ADE
:100246007BFF7A11795290668DE0F52D12144A7B68
:10025600FF7A1179859062B6E0F52D12144A7BFF7C
:100266007A1179B3A201E433F52D12144A7BFF7A91
:100276001179DF90667DE0F52DA3E0F52EA3E0F57C
:100286002FA3E0F530A3E0F531A3E0F53212144ACE
:100296001231427BFF7A12792A12144A229063782D
:1002A600E0644C70527E127F30122648906380E0E4
:1002B600F525A3E0F526E4F5277D03AF26AE251246
:1002C60027297E127F6B122648AE25AF26E4FB7DDA
:1002D600101228037E127F6E12264874102526F50A
:1002E60026E43525F5250527E527C3941040CA7E63
:1002F600127F6E12264822906378E0646C705CF57B
:10030600297E127F70122648E4F528AF297E007DEB
:10031600031227297E127F6B122648E4F527A829A7
:10032600E6FF74822527F582E43463F583EFF00552
:10033600290527E527B410E67E637F82E4FB7D105E
:100346001228037E127F6E1226480528E528C394DC
:100356000840B87E127F6E12264822906378E064C9
:100366004B7061F527746A2527F582E43463F583BB
:10037600E06032746A2527F582E43463F583E0F49D
:100386006023746A2527F582E43463F583E0FF74FD
:10039600802527F582E43463F583E0B50710052749
:1003A600E527B408C09061047432F00208779063C0
:1003B600787421F0300A030208777E127FAB12268A
:1003C60048020877906378E0B4521A200A077E1232
:1003D6007FB31226489063787472F07E637F787DCF
:1003E60008122C6722906378E064497045200A075A
:1003F6007E127FBE122648906380E0F525A3E0F5C5
:1004060026E4F527852682852583E0FF7482252745
:10041600F582E43463F583EFF00526E526700205E0
:10042600250527E527B480DC7E637F787D8A122C3C
:100436006722906378E064437079A3E06452704663
:10044600200A077E127FC6122648906380E0F525B3
:10045600A3E0F526E4F527852682852583E493FF28
:1004660074822527F582E43463F583EFF00526E5EB
:1004760026700205250527E527B480DB7E637F7895
:100486007D8A122C6722906379E064576003020824
:1004960080906380E0F525A3E0F52674822527F594
:1004A60082E43463AD82FC7B80AF26AE25123255E2
:1004B600020877906378E06444600302054A90631B
:1004C60080E0FF64447003020877EFB4310CC20A7F
:1004D6007E127FCF122648020877906380E0B43000
:1004E6000CD20A7E127FDB122648020877906380C0
:1004F600E0B4320CD20B7E127FE81226480208774F
:10050600906380E0B4330CC20B7E127FF61226484D
:10051600020877906380E0B4340CD20C7E137F051A
:10052600122648020877906380E0B4350CC20C7E30
:10053600137F12122648020877906380E0FF123379
:10054600AB020877906104E07013200A077E137FE0
:10055600201226489063787421F00208779061048F
:100566007432F0906378E0FFB4510A908000748092
:10057600F0C2AF80FEEF64577045200A077E137FF6
:100586002E122648906381E0906334F0E4F52790BC
:100596006334E0FFE527C39F400302087774822592
:1005A60027F582E43463F583E0FF906380E0252736
:1005B60024AFF582E43461F583EFF0052780D0900F
:1005C6006378E064536003020679200A077E137F8E
:1005D60039122648906341E0FF9061B8E06F703CA5
:1005E600906342E0FF9061B9E06F7030906343E042
:1005F600FF9061BAE0B50724906344E0FF9061BBC9
:10060600E0B50718906345E0FF9061BCE0B5070CC4
:10061600906346E0FF9061BDE06F6016906378746A
:1006260021F0300A030208777E137F48122648021B
:100636000877E4F527E4F518AF27FE74AF2527F50C
:1006460082E43461F583E0FD1233700527E527C3A4
:1006560094FE40E19080007480F0C2AFE4907FF099
:10066600F0A3F0907FFD74AAF0A374FFF0A3745575
:10067600F080FE906378E0644F704C906380E0F504
:1006860025A3E0F526E5264525700A200A077E13F0
:100696007F51122648200A077E137F58122648E407
:1006A600F52774822527F582E43463F583E08526F1
:1006B60082852583F00526E526700205250527E5B2
:1006C60027B480DE020877906378E0FFB445279070
:1006D60080007480F0906380E0FDA3E0907FF0CD11
:1006E600F0A3EDF0C2AF907FFD74AAF0A374FFF003
:1006F600A37455F080FEEF6465600302087790638B
:1007060080E0FFA3E0907FF0CFF0A3EFF0E4F525C3
:10071600F526D3907FF1E09526907FF0E095254071
:1007260020E4F5182526FFE5253401FE8526828579
:100736002583E0FD1233700526E526700205258027
:10074600D17E137F5A122B5EEF4E6020120003906B
:100756006347EFF0120003906348EFF01200039036
:100766006349EFF012000390634AEFF07E137F6057
:10077600122B5EEF4E6020120003906350EFF012D2
:100786000003906351EFF0120003906352EFF012F2
:100796000003906353EFF07E137F66122B5EEF4EDD
:1007A6006020120003906354EFF01200039063552B
:1007B600EFF0120003906356EFF0120003906357B8
:1007C600EFF07E137F6C122B5EEF4E60201200035B
:1007D60090633DEFF012000390633EEFF0120003CA
:1007E60090633FEFF0120003906340EFF07E137FBB
:1007F60072122B5EEF4E6020120003906339EFF009
:1008060012000390633AEFF012000390633BEFF09F
:1008160012000390633CEFF07E137F78122B5EEF9D
:100826004E6008123033906358EFF0E4F527E4F594
:1008360018E5272401FFE433FE74392527F582E401
:100846003463F583E0FD1233700527E527C394432F
:1008560040DC9080007480F0C2AFE4907FF0F0A39B
:10086600F0907FFD74AAF0A374FFF0A37455F08096
:0A087600FE7E637F787D08122C6778
:010880002255
:10321D00AE07EEC39430400BEED394395005EE2437
:10322D00D0FF22EEC39461400BEED394665005EEB1
:10323D0024A9FF22EEC39441400BEED394465005D2
:08324D00EE24C9FF22AF0622A6
:103356009062AFE004F070069062AEE004F0906216
:0A336600AEE0FEA3E0FF12333A22AE
:1000030012335612321DEFC454F0FEC0061233569B
:0800130012321DD0E02FFF2284
:10303300E49068AFF01233569068B0EFF0C3943069
:103043004018E0FFD3943950119068AFE02407F59E
:1030530082E43461F583EFF080119068AFE02407D8
:10306300F582E43461F583E4F0800C9068AFE0040A
:10307300F0E0D3940840BE752D00752E00752F0027
:0C308300E4F5307B017A617907121D6CC6
:01308F00221E
:042B5E008E2A8F2B01
:102B62009062AEE4F0A374FFF0123356EF606EF49D
:102B7200606B852B82852A83E493B507EC752C0163
:102B8200E52B252CF582E4352AF583E49360259024
:102B920062AFE0252CFF9062AEE03400FE12333AC1
:102BA200E52B252CF582E4352AF583E493B5070459
:102BB200052C80CCE52B252CF582E4352AF583E41F
:102BC2009370A6E52C24FFFFE434FFFE9062AFE091
:102BD2002FF09062AEE03EF07E007F0122E4FEFF25
:012BE20022D0
:102562007E137FA9122B5EEF4E70037F01227E1332
:102572007FAC122B5EEF4E600C123356EF24D02448
:10258200FF920E8002D20E7E137FB2122B5EEF4EAE
:10259200600C123356EF24D0906683F08005E490ED
:1025A2006683F07E137FB8122B5EEF4E600C1233FF
:1025B20056EF24D090668DF08005E490668DF07E13
:1025C200137FBE122B5EEF4E600C123356EF24D0F7
:1025D2009062B6F08005E49062B6F07E137FC4127A
:1025E2002B5EEF4E600C123356EF24D024FF920183
:1025F2008002C20190634163A20190667D63A201E1
:102602007F06121C9530013B7E137FCA122B5EEFB0
:102612004E603012000390667DEFF0120003906668
:102622007EEFF012000390667FEFF01200039066D7
:1026320080EFF0120003906681EFF01200039066C3
:0626420082EFF07F002290
:1019C700C201E490668DF0D20EC204906683F09057
:1019D70062B6F090634163A20190667D63A2017FC6
:1019E70006121C95E4F525E52575F003A424D0F52A
:1019F70082E43413F583E493FB740193FA7402933E
:101A0700F91217447003021BB9E4F526F527FD7494
:101A17002F2DF582E43461F583E0FF7003021BB4D8
:101A2700E52575F003A424D0F582E43413F583E4A7
:101A370093FB740193FA740293F9852682758300E8
:101A470012175DFEEFB506087527010526021BB0C4
:101A5700E5277003021BB0EE6003021BABE52524EC
:101A6700FE6028147003021B93147003021B971463
:101A77007003021B9F147003021BA324056003025B
:101A87001BB490668D7401F0021BB4D201742F2D24
:101A9700F582E43461F583E0FF642D7003021BB423
:101AA70012321DEFC454F0FC74302DF582E434611A
:101AB700F583E0FF12321DEF2C90667DF074312D17
:101AC700F582E43461F583E0FF12321DEFC454F070
:101AD700FC74322DF582E43461F583E0FF12321D88
:101AE700EF2C90667EF074332DF582E43461F58334
:101AF700E0FF12321DEFC454F0FC74342DF582E47C
:101B07003461F583E0FF12321DEF2C90667FF0748D
:101B1700352DF582E43461F583E0FF12321DEFC401
:101B270054F0FC74362DF582E43461F583E0FF123E
:101B3700321DEF2C906680F074372DF582E4346106
:101B4700F583E0FF12321DEFC454F0FC74382DF515
:101B570082E43461F583E0FF12321DEF2C90668139
:101B6700F074392DF582E43461F583E0FF12321DFC
:101B7700EFC454F0FC743A2DF582E43461F583E048
:101B8700FF12321DEF2C906682F08021D204801D57
:101B97009066837401F08015C20E80119062B6744E
:101BA70001F08009E4F527F5260D021A160525022E
:021BB70019EE25
:011BB9002209
:10319A00906579E0C3947C503D906579E0FE04F037
:1031AA0074B72EF582E43462F583EFF0BF0A2790F4
:1031BA006579E0FF04F074B72FF582E43462F58391
:1031CA00E4F0906579E0FF122CE99065797408F0D3
:0731DA009062B8E004F0224E
:103090009080007480F090633963A201F583F5821B
:1030A00063A2017F08121C9590634163A201908086
:1030B0008863A2017F0A121C95908092E4F0A374A9
:1030C00032F0A37401F090634BE0FF9080B1F09078
:1030D00080E1EFF09080957455F0A3F0908000743B
:0930E00001F09080097470F022E7
:102EDC00908009E04410F09080A0E0706C9080A18C
:102EEC007482F09080A874FFF0A3F0A3F0A3F07F9D
:102EFC00039080AEEFF07FCBA3EFF07F039080AC1C
:102F0C00EFF0A374CBF09080007402F09068A312E1
:102F1C001895000000009068A3E0908040F0906845
:102F2C00A4E0908041F09068A5E0908042F0906819
:102F3C00A6E0908043F0A3E4F0A3F0A3F0A3F090FC
:092F4C008018F0A3F0A3F0A3F03B
:012F55002259
:102FD000908009E04440F09080D17482F090634C7E
:102FE000E0FF9080DEF090634DE0FF9080DFF09096
:102FF00080027402F09068A71218950000000090FB
:1030000068A7E0908058F09068A8E0908059F09010
:1030100068A9E090805AF09068AAE090805BF0A3E5
:10302000E4F0A3F0A3F0A3F0908030F0A3F0A3F0BD
:02303000A3F00B
:01303200227B
:102F5600908009E04420F09080B8E0706C9080B9D1
:102F66007482F07F039080C6EFF07FCDA3EFF07FF1
:102F7600039080C4EFF0A374CDF09080C074FFF08E
:102F8600A3F0A3F0A3F09080017402F09068AB1256
:102F96001895000000009068A7E090804CF09068BB
:102FA600A8E090804DF09068A9E090804EF090687F
:102FB600AAE090804FF0A3E4F0A3F0A3F0A3F09072
:092FC6008024F0A3F0A3F0A3F0B5
:012FCF0022DF
:102BE3008C258D26A907EAFDE975F018A424ACFF0E
:102BF300E5F034808F82F583EDF0EBFDE975F01895
:102C0300A4FFAEF024ACFBEE34808B82F583A3EDFE
:102C1300F08526828C83E0FDEF24A8FFEE3480FE4E
:102C23008F82F583EDF08526828C83A3E08F828EDD
:102C330083A3F0852682852583A3A3E0FDE975F0B0
:102C430018A424A8FFE5F03480FE8F82F583A3A3A4
:102C5300EDF08526828C83A3A3A3E08F828E83A3CA
:042C6300A3A3F02215
:062C67008D2AAB07AA064E
:102C6D009068A3E0FCA3E0FDA3E0FEA3E0F52E8EAB
:102C7D002D8D2C8C2BAE02AF038E838F8263A20120
:102C8D00E52D540744C0F583852E8263A201AF2A3A
:102C9D00121CFE908000E020E5F9E4FCFDFEE52E1F
:102CAD00252AF52EEE352DF52DED352CF52CEC35A3
:102CBD002BF52B908040E52BF0A3E52CF0A3E52D13
:102CCD00F0A3E52EF09080007420F0AF2EAE2DAD68
:0B2CDD002CAC2B9068A3121889AF2AC2
:012CE80022C9
:062E61008D25AB07AA0657
:102E67009068A7E0FCA3E0FDA3E0FEA3E0F5298EB0
:102E7700288D278C26AE02AF038E838F8263A20133
:102E8700E528540744D0F58385298263A201AF253D
:102E9700121CFEE4FCFDFEE5292525F529EE352863
:102EA700F528ED3527F527EC3526F526908058E5EA
:102EB70026F0A3E527F0A3E528F0A3E529F0908005
:102EC700027420F0AF29AE28AD27AC269068A71270
:042ED7001889AF2582
:012EDB0022D4
:02298C008F2595
:10298E00908001E030E5037F00229068ABE0FCA36D
:10299E00E0FDA3E0FEA3E0F5298E288D278C26907E
:1029AE00667D63A201E528540744C8F58385298214
:1029BE0063A2017F06121D14E5292406F529E435CC
:1029CE0028F528E43527F527E43526F52690657B8E
:1029DE0063A201E528540744C8F58385298263A2C2
:1029EE0001AF25121D14E4FCFDFEE5292525F52970
:1029FE00EE3528F528ED3527F527EC3526F526900A
:102A0E00804CE526F0A3E527F0A3E528F0A3E52901
:102A1E00F09080017420F0AF29AE28AD27AC26903F
:072A2E0068AB121889AF2507
:012A3500227E
:10245E009081E0E0F52505250525052505250525B1
:10246E0005250525052505250525908010E0F5286F
:10247E00A3E0F529A3E0F52AA3E0F52B9081E1E096
:10248E00F5250525052505250525052505250525FE
:10249E00052505250525908014E0F52CA3E0F52DE6
:1024AE00A3E0F52EA3E0F52FE52EB52A08E52FB50E
:1024BE002B037F0022E4F525E52E540744E0F58337
:1024CE00852F8263A20190637863A2017F08121D9B
:1024DE002C90637A63A2019062B063A2017F061210
:1024EE001C95906378E0F526A3E0F527E4F525909A
:1024FE006378E0702AA3E024F8F525E52E5407440E
:10250E00E0F583852F8274082582F582E43583F504
:10251E008363A20190637863A201AF25121D2CAED6
:10252E0026E4FCFDE52F2527F52FE52E3EF52EEDB5
:10253E00352DF52DEC352CF52C908014E52CF0A3D3
:10254E00E52DF0A3E52EF0A3E52FF090800074406A
:03255E00F0AF25B6
:012561002257
:101F10009081E6E0F52505250525052505250525FE
:101F200005250525052505250525908028E0F528AA
:101F3000A3E0F529A3E0F52AA3E0F52B9081E7E0E3
:101F4000F525052505250525052505250525052551
:101F500005250525052590802CE0F52CA3E0F52D21
:101F6000A3E0F52EA3E0F52FE4F525E52EB52A0A2A
:101F7000E52FB52B05C20802206AE52E540744F070
:101F8000F583852F8263A20190637863A2017F08A5
:101F9000121D2C906378E0F526A3E0F527E5274590
:101FA0002670099080027410F07F0022906684E011
:101FB000FFF4602D90637AE06F7076906685E0FFA5
:101FC00090637BE06F706A906686E0FF90637CE0D0
:101FD0006F705E906687E0FF90637DE06F602280A7
:101FE0005090637AE0906684F090637BE090668521
:101FF000F090637CE0906686F090637DE090668769
:10200000F0906378E0702AA3E024F8F525E52E54DB
:102010000744F0F583852F8274082582F582E43524
:1020200083F58363A20190637863A201AF25121D3B
:102030002CAE26E4FCFDE52F2527F52FE52E3EF5F9
:102040002EED352DF52DEC352CF52CAF2BAE2AAD24
:1020500029AC28AB2FAA2EA92DA82CD31218784072
:10206000099080027410F07F002290802CE52CF003
:10207000A3E52DF0A3E52EF0A3E52FF090800274E8
:0420800040F0AF2558
:012084002239
:102085009081E3E0F525052505250525052505258B
:102095000525052505250525052590801CE0F52840
:1020A500A3E0F529A3E0F52AA3E0F52B9081E4E070
:1020B500F5250525052505250525052505250525DB
:1020C500052505250525908020E0F52CA3E0F52DB7
:1020D500A3E0F52EA3E0F52FE4F525E52EB52A0AB4
:1020E500E52FB52B05C2090221D0E52E540744E89A
:1020F500F583852F8263A20190600463A2017F0EA0
:10210500121D42906004E0F526A3E0F52790600CCF
:10211500E0FFF4604590667DE0FEEF6E706EA3E033
:10212500FF90600DE06F706490667FE0FF90600E39
:10213500E06F7058906680E0FF90600FE06F704C24
:10214500906681E0FF906010E06F7040906682E0DD
:10215500FF906011E06F60048032D2D9906004E096
:10216500702AA3E024F2F525E52E540744E8F5830B
:10217500852F82740E2582F582E43583F58363A26B
:102185000190600463A201AF25121D42AE26E4FC56
:10219500FDE52F2527F52FE52E3EF52EED352DF501
:1021A5002DEC352CF52CAF2BAE2AAD29AC28AB2F59
:1021B500AA2EA92DA82CD31218785006E527452656
:1021C50070099080017410F07F0022908020E52C2A
:1021D500F0A3E52DF0A3E52EF0A3E52FF090800107
:0521E5007440F0AF257D
:0121EA0022D2
:042648008E2A8F2B1C
:10264C009068A3E0FCA3E0FDA3E0FEA3E0F5318ECF
:10265C00308D2F8C2EE531FFE5305407FEE42FF53D
:10266C002DEE34C0F52C852D82F5837423F0052DC9
:10267C00E52D7002052C532CC7F582852C83740A2A
:10268C00F0052DE52D7002052C532CC7906341638A
:10269C00A201852C83852D8263A2017F06121CFE6C
:1026AC007406252DF52DE4352CF52C852A83852BE8
:1026BC008263A201852C83852D8263A201121CE208
:1026CC00908000E020E5F9E4FCFDFE9068A3E0F8C2
:1026DC00A3E0F9A3E0FAA3E02FFFEE3AFEED39FDFB
:1026EC00EC38FCEF2408FFE43EFEE43DFDE43CFC4A
:1026FC009068A31218899068A3E0908040F09068CD
:10270C00A4E0908041F09068A5E0908042F0906841
:0C271C00A6E0908043F09080007420F054
:01272800228E
:062803008E2A8F2B8D2CA4
:102809009068A3E0FCA3E0FDA3E0FEA3E0F5328E0F
:10281900318D308C2FE532FFE5315407FEE42FF579
:102829002EEE34C0F52D852E82F5837423F0052E06
:10283900E52E7002052D532DC7F582852D83EBF00A
:10284900052EE52E7002052D532DC790634163A215
:1028590001852D83852E8263A2017F06121CFE74D9
:1028690006252EF52EE4352DF52D852A83852B8217
:1028790063A201852D83852E8263A201AF2C121CD0
:10288900FE908000E020E5F97408252CF52CFFE482
:10289900FCFDFEE5322FF532EE3531F531ED3530FF
:1028A900F530EC352FF52F908040E52FF0A3E5307A
:1028B900F0A3E531F0A3E532F09080007420F0AF89
:0D28C90032AE31AD30AC2F9068A3121889EB
:0128D60022DF
:022CE9008F3E1C
:102CEB009068A3E0FCA3E0FDA3E0FEA3E0F5428E19
:102CFB00418D408C3FE542FFE5415407FEE42FFF39
:102D0B00EE34C09062B763A201F5838F8263A20198
:102D1B00AF3E121CFE908000E020E5F9E4FCFDFEC6
:102D2B00E542253EF542EE3541F541ED3540F540A6
:102D3B00EC353FF53F908040E53FF0A3E540F0A335
:102D4B00E541F0A3E542F09080007420F0AF42AE75
:0B2D5B0041AD40AC3F9068A312188906
:012D6600224A
:062729008E2A8F2BAB0588
:10272F009068A3E0FCA3E0FDA3E0FEA3E0F5318EEB
:10273F00308D2F8C2EE531FFE5305407FEE42FF559
:10274F002DEE34C0F52C852D82F5837423F0052DE5
:10275F00E52D7002052C532CC7F582852C83EBF0E9
:10276F00052DE52D7002052C90634163A201852C88
:10277F0083852D8263A2017F06121CFE7406252D10
:10278F00F52DE4352CF52C532CC7E52A852D8285A4
:10279F002C83F0052DE52D7002052C532CC7F582E7
:1027AF00852C83E52BF0052DE52D7002052C532C80
:1027BF00C7908000E020E5F9E531240AF531E435D2
:1027CF0030F530E4352FF52FE4352EF52E9080407F
:1027DF00E52EF0A3E52FF0A3E530F0A3E531F0905F
:1027EF0080007420F0AF31AE30AD2FAC2E9068A3C7
:0327FF0012188924
:0128020022B3
:10333A00E5D220E0FBC2AF438E2075D2028F828E87
:0B334A0083E0FFE4F5D2538EDFD2AF2A
:013355002255
:10337000E5D220E0FBC2AF43D2028F828E83EDF014
:0933800075D25063D250D2AF2285
:102D6700E4FDED2401FFE433FE12333A74392DF507
:102D770082E43463F583EFF00DBD3FE6E4FDED2417
:102D87007FFFE433FE12333A742F2DF582E434616A
:102D9700F583EFF0742F2DF582E43461F583E0704D
:102DA7001B742F2DF582E43461F5837420F07430A1
:102DB7002DF582E43461F583E4F080040DBD80BE17
:102DC700E49061AEF0FDEDFF7E0012333A74AF2D53
:0D2DD700F582E43461F583EFF00DBDFEE9F7
:012DE40022CC
:023255008B2AC2
:10325700A2AF920FC2AF85A22B53A2FE8E838F829D
:1032670005A28C838D827409121D5AE52A53A2FE8A
:1032770043A220121D5C53A2DF852BA2A20F92AF9F
:01328700FF47
:013288002223
:10330100A2AF920FC2AF8C838D82EF121D5A43A2DE
:0C33110020121D5C53A2DFA20F92AFFF40
:01331D00228D
:0232B9008F255F
:1032BB00A2AF920FC2AFE4F5838D827406121D5A32
:1032CB00E52543A220121D5C53A2DFA20F92AF7F14
:0132DB0001F1
:0132DC0022CF
:0232DD008F253B
:1032DF00A2AF920FC2AFE4F5838D82740A121D5A0A
:1032EF00E52543A220121D5C53A2DFA20F92AF7FF0
:0132FF0001CD
:0133000022AA
:101BBA00A907E7FFA805EF93C3966008403B74FCAA
:101BCA002FFF80F00F08EF93C3966008402B74FB39
:101BDA002FFF80E00F08EF93C3966008401B74FA4A
:101BEA002FFF80D00F08EF93D3966008400B74F94B
:101BFA002FFF80C01F1F1F1F1FEF54FEF80303F79C
:101C0A00E893FC08E893FD08E893FE08E893FF22AE
:101C1A0009E993C39D6008402974FB29F980F109F9
:101C2A00E993C39E6008401A74FA29F980E209E927
:101C3A0093D39F6008400B74F929F980D3191919B5
:101C4A001919E9C313C313FF22740093F8ECC3985C
:101C5A004024701F740193F8EDC3984019701474EE
:0E1C6A000293F8EEC398400E7009740393F8CD
:101C7800EFC39840037F00227F0122EDF8E6F008C9
:101C8800A3DFFA22EDF8E0F608A3DFFA22E0A36367
:101C9800A201F0A363A201DFF475A20022E0A3630E
:101CA800A201F0A363A201E0A363A201F0A363A2CF
:101CB80001E463A201F0A363A201DFE175A200229F
:101CC800E0A363A2016DFE936CFDEE058393FC1502
:101CD8008363A201DFEA75A200227F00E493A36375
:101CE800A201F00F600CA3E583C2E3F58363A201B0
:101CF80080EA75A20022E0A363A201F0A3E583C2F3
:101D0800E3F58363A201DFEE75A20022E0A363A2DC
:101D180001F0A3E583C2E4D2E3F58363A201DFEC1B
:101D280075A20022E583C2E3F583E0A363A201F074
:101D3800A363A201DFEE75A20022E583C2E4D2E329
:101D4800F583E0A363A201F0A363A201DFEC75A20F
:101D58000022F922C002C004C00612FFF0D006D04B
:041D680004D002227F
:102338003E2A2C312CCFE0F0E0ECE5F2F0FB20EE69
:10234800E1ECE5EDE020F120C8C2D72D310A003ECE
:102358004C2C4930312C256C752CD1EAEEF0EEF17D
:10236800F2FC20EEE1ECE5EDE02C35302C3130309C
:102378002C3330302C3630302C313230302C323453
:1023880030302C343830302C393630302C3139322A
:1023980030302C33383430302C35373630302C311F
:1023A80031353230300A003E422C4930322C256219
:1023B800752CC2FBF1F2E0E2EBFFF2FC2052545321
:1023C80020EFF0E820EFE5F0E5E4E0F7E50A003E6D
:1023D800532C5630382C2562752CC8EDF2E5F0E206
:1023E800E0EB20EEEFF0EEF1E020F7E0F1F2EEF2B4
:1023F800FB282A3130ECF1290A003C21003C493005
:10240800313D003C4930323D003C5630383D000AF1
:10241800C7E0EFF0EEF120F7E0F1F2EEF2FB0A0090
:10242800CEF8E8E1EAE020CAD1210A00CFF0E8EDD1
:10243800FFF2EE3A00203EC2F0E5ECFF202562757F
:102448003A2562753A2562752020F7E0F1F2EEF23E
:06245800E02025750A00DA
:1033240052668F0000000000000000000000000052
:05333400000000000094
:0133AB0022FF
:030023000232891D
:10328900C0E0C083C082C0D0309817751601D291B2
:1032990074A1250BF582E43466F583E599F0050BF5
:1032A900C298309902C299D0D0D082D083D0E0326E
:103142007BFF7A23793812144A9068A1E0FEA3E04B
:10315200FFC3E49FFFE49EFEAB07FA3395E0F9F864
:103162007F007E8C7D0A7C001217D88F308E2F8DC7
:103172002E8C2D7BFF7A23795712144A7BFF7A23F8
:1031820079AFA21AE433F52D12144A7BFF7A237920
:08319200D785122D12144A2208
:102DE5007E247F02122B5EEF4E70037F01227E242C
:102DF5007F05122B5EEF4E6023123033A804A90520
:102E0500AA06AB077F007E8C7D0A7C001217D812BC
:102E1500186A9068A1EEF0A3EFF0800A9068A1749B
:102E2500FFF0A374B8F07E247F0B122B5EEF4E608B
:102E35000C123356EF24D024FF921A8002C21A7E58
:102E4500247F11122B5EEF4E60091230338E118FE5
:0C2E55001280067511007512647F0022C7
:1030E900C219C21CE4F50BF516D296C21BF50FF5F1
:1030F90010750C05F508F509122DE5C2ADE4F5C901
:10310900D2CDD2CCC2C9C2CAF5CDF5CC9068A1E066
:10311900F5CBA3E0F5CA85CBCD85CACCE4F598D229
:103129009E438740C29FC2ACC298C29975B81075B8
:09313900B710D2CAD29CD2AC221C
:0133AC0022FE
:1028D700E4FF0F2407F582E43461F583E50DF00F7B
:1028E70074072401F582E43461F583E4F07C667DA6
:1028F70094FEED1DAA0470011CF5828A83E0FBAAF1
:10290700070F74072AF582E43461F583EBF00EBEF6
:1029170004E07C667D98E4FEED1DAA0470011CF5B9
:10292700828A83E0FBAA070F74072AF582E43461E1
:10293700F583EBF00EBE04E07C667D9CE4FEED1DA6
:10294700AA0470011CF5828A83E0FBAA070F7407AB
:102957002AF582E43461F583EBF00EBE04E07C6671
:102967007DA0E4FEED1DAA0470011CF5828A83E0B8
:10297700FBAA070F74072AF582E43461F583EBF0AD
:042987000EBE04E09C
:01298B002229
:05001E00D29CD2AC22CF
:0333A800D21C2212
:1031E100E510450F6033E4906478F0A37407F09024
:1031F100667CE090647AF0A37411F0A37402F0A3EA
:1032010014F0A3F0E4A3F0A3E510F0E50FA3F0E4BC
:0C321100A3F0F50FF5107F01227F0022D2
:0133AD0022FD
:1021EB0030020A0509E50970020508C202D3E509A8
:1021FB009512E5089511401C12001EC291A290B3D6
:10220B009290E4F508F509759963200A077E247FFF
:10221B0017122648E50BD394005003022337E5161B
:10222B00D3950C5003022337C291850B0EE4F50BAB
:10223B00F516FF7E02E50E14FDEEC39D501074A142
:10224B002EF582E43466F583E02FFF0E80E774A051
:10225B00250EF582E43466F583E06F600E300A03D9
:10226B000223377E247F28122648229066A1E06441
:10227B006370609066A9E0F9FFE4C4F854F0C86895
:10228B00FEEFC4540F48FF7C037DE812178AAA06A1
:10229B00AB079066A8E07E00540FFF7C277D1012E1
:1022AB00178AEF2BFDEE3AFCE9540F75F064A42D61
:1022BB00FDE5F03CFC9066AAE0FBC4540F75F00AF8
:1022CB00A42DFFE5F03CFEEB540F7C002FF510EC3A
:1022DB003EF50F200A567E247F341226487E667FF9
:1022EB00A1E4FBAD0E1228037BFF7A24793D9066A7
:1022FB00A3E0FFC4540F75F00AA4FEEF540F2EF5A4
:10230B002DA3E0FFC4540F75F00AA4FEEF540F2E5B
:10231B00F52EA3E0FFC4540F75F00AA4FEEF540F83
:0C232B002EF52F850F3085103112144A5A
:012337002283
:0B339D00301C05C21C7F01227F0022B3
:102ADE00020881E493A3F8E493A34003F68001F285
:102AEE0008DFF48029E493A3F85407240CC8C333F9
:102AFE00C4540F4420C8834004F456800146F6DFC8
:102B0E00E4800B010204081020408090331EE47E06
:102B1E00019360BCA3FF543F30E509541FFEE493BC
:102B2E00A360010ECF54C025E060A840B8E493A383
:102B3E00FAE493A3F8E493A3C8C582C8CAC583CAAE
:102B4E00F0A3C8C582C8CAC583CADFE9DEE780BE66
:013339000093
:10174400BB010689828A83E0225002E722BBFE02A3
:09175400E32289828A83E49322D6
:10175D00BB010CE58229F582E5833AF583E0225041
:10176D0006E92582F8E622BBFE06E92582F8E2228B
:0D177D00E58229F582E5833AF583E49322A5
:10178A00EF8DF0A4A8F0CF8CF0A428CE8DF0A42E73
:02179A00FE222D
:10179C0075F008758200EF2FFFEE33FECD33CDCC04
:1017AC0033CCC58233C5829BED9AEC99E582984087
:1017BC000CF582EE9BFEED9AFDEC99FC0FD5F0D664
:1017CC00E4CEFBE4CDFAE4CCF9A88222B800C1B98E
:1017DC000059BA002DEC8BF084CFCECDFCE5F0CBCC
:1017EC00F97818EF2FFFEE33FEED33FDEC33FCEB05
:1017FC0033FB10D703994004EB99FB0FD8E5E4F9C0
:10180C00FA227818EF2FFFEE33FEED33FDEC33FCAC
:10181C00C933C910D7059BE99A4007EC9BFCE99AA0
:10182C00F90FD8E0E4C9FAE4CCFB2275F010EF2FE5
:10183C00FFEE33FEED33FDCC33CCC833C810D707E5
:10184C009BEC9AE899400AED9BFDEC9AFCE899F820
:0E185C000FD5F0DAE4CDFBE4CCFAE4C8F922B3
:0E186A00C3E49FFFE49EFEE49DFDE49CFC228F
:10187800EB9FF5F0EA9E42F0E99D42F0E89C45F0C6
:01188800223D
:0C188900ECF0A3EDF0A3EEF0A3EFF022D2
:10189500A8828583F0D083D0821218AC1218AC12BE
:1018A50018AC1218ACE473E493A3C583C5F0C583E3
:1018B500C8C582C8F0A3C583C5F0C583C8C582C89D
:0118C5002200
:1013E800E539242DF8E6053922782A301602782DB9
:1013F800E475F001121927021744200FEB7F2ED253
:101408000F8018EF540F2490D43440D4FF30130BBE
:10141800EF24BFB41A0050032461FFE53A600215B7
:101428003A053DE53D7002053C30160D782AE47515
:10143800F001121927EF0218C602319A7403D21666
:101448008003E4C216F5398B2A8A2B892CE4F53AF5
:10145800F53CF53DE53A60077F2012142380F575C9
:101468003BFFC210C20FC211C212C214C215C2176A
:101478001213F1FF700D3016057F00121434AF3DC2
:10148800AE3C22B4255FC2D5C2131213F1FF24D09B
:10149800B40A00501A75F00A783A30D50508B6FF34
:1014A8000106C6A426F620D5047002D21280D924DB
:1014B800CFB41A00EF5004C2E5D213021634D2108A
:1014C80080C6D20F80C0D21180BCD2D580BAD214C7
:1014D80080B47F201214232011077401B53A00400C
:1014E800F11213E8FF12142302145CD217D21580EC
:1014F800951213E8FB1213E8FA1213E8F94A4B7035
:101508000679057A177BFF20112EE53A602A7E00BE
:101518008E8275830012175D60060EEE653B70F0D3
:10152800C2D5EBC0E0EAC0E0E9C0E0EE12167BD01D
:10153800E0F9D0E0FAD0E0FB121744FF60AAEBC054
:10154800E0EAC0E0E9C0E0121423D0E02401F9D0B9
:10155800E03400FAD0E0FBE53B0460DCD53BD98001
:10156800877BFF7A167977D211809C79108002796F
:1015780008C215C2178008D2D5790A8004790AC230
:10158800D5E53B047002F53BE4FAFDFEFF1213E8D3
:10159800FC7B082010131213E8FD7B10300F0A1291
:1015A80013E8FE1213E8FF7B20EC3382D592D55066
:1015B80013C3E4300F069FFFE49EFEE42010039D52
:1015C800FDE49CFCE4CBF8C210EC700CCFCECDCC83
:1015D800E824F8F870F38017C3EF33FFEE33FEED1D
:1015E80033FDEC33FCEB33FB994002FB0FD8E9EBFE
:1015F800301005F8D0E0C448B210C0E00AEC4D4EF7
:101608004F78207B0070C2EAB53B0040BCC0E012B6
:10161800167DD0F0D0E0201004C4C0E0C4B210C0E1
:10162800F012140CD0F0D5F0EB02145C12198614E9
:10163800F95315735814CA4C14C64215774F157FC1
:0F16480044157F4914DF4315855515694615690B
:101657004515694717255014CE2D14D22E14F52B96
:1016670014D62314F320170E2A148E48000014ED05
:101677003F3F3F00790AA2D5201214301409B91050
:10168700020404B9080104A2D52015025001042060
:1016970011689211B53A005034C0E07F203012191A
:1016A7007F30A21172157214500F1216D4C211C2D4
:1016B70015C214C2177F30800F301403E9C0E0123F
:1016C7001423301403D0E0F9D0E0B53ACC30141726
:1016D7007F30B9100C1214237F583013077F78809E
:1016E70003B908031214233011057F2D0214237F39
:1016F700202017F87F2B2015F322921180CF286E18
:10170700756C6C2900D2101213E83010F8C21078EB
:101717003A30D50108F602148E2D5043495812135A
:10172700E82403B405004001E49017209312141431
:0D173700743A121414D212753A040215739C
:101D6C008B2A8A2B892CE4F536F535F534F533F5C9
:101D7C0031F532E52E452F452D6012EBC0E0EAC05F
:101D8C00E0E9C0E0AB2DAA2EA92F121937AB2A051A
:101D9C002CE52CAA2B7002052B14F9121744F537DD
:101DAC00C394094007E537D3940D40E1E53764202F
:101DBC0060DBE537B42D054332038016E537B42BD1
:101DCC0005433201800C74FF252CF52C74FF352B48
:101DDC00F52BE53060046410703FAB2AAA2BA92CBC
:101DEC0012174464306009E530702E75300A802972
:101DFC0090000112175DFF64786004EFB458134330
:101E0C0032017530107402252CF52CE4352BF52B92
:101E1C008007E5307003753008AB2A052CE52CAA39
:101E2C002B7002052B14F9121744F537C39461403B
:101E3C000AE537D3947A50035337DF74D02537F53E
:101E4C0037C3940A400CE5379411406D74F925376B
:101E5C00F537E537D39530506043320185363B85F5
:101E6C00353A853439853338AF307E00E4FCFDAB30
:101E7C0036AA35A934A8331218D8C8ECC8C9EDC98C
:101E8C00CAEECACBEFCBE4FCFDFEEB2537F536EE04
:101E9C003AF535ED39F534EC38F533AF36AE35ADC2
:101EAC0034FCAB3BAA3AA939A838D31218785003A2
:101EBC00021E25433204021E25E53220E003E48095
:101ECC002DE52E452F452D601EAB2AE52C24FFF960
:101EDC00E52B34FFFAEBC0E0EAC0E0E9C0E0AB2D43
:101EEC00AA2EA92F121937E53230E20774FFFFFE34
:101EFC00FDFC22E532AF36AE35AD34AC3330E10308
:041F0C0002186A222B
:1018C600BB010689828A83F0225002F722BBFE0101
:0218D600F322FB
:1018D800E88FF0A4CC8BF0A42CFCE98EF0A42CFCAF
:1018E8008AF0EDA42CFCEA8EF0A4CDA8F08BF0A42D
:1018F8002DCC3825F0FDE98FF0A42CCD35F0FCEB8C
:101908008EF0A4FEA9F0EB8FF0A4CFC5F02ECD3950
:0F191800FEE43CFCEAA42DCE35F0FDE43CFC22BD
:10192700FAE6FB0808E6F925F0F618E6CA3AF622C1
:10193700BB011A89828A83D0F0D0E0F8D0E0F9D0D1
:10194700E0FAD0E0FBE8C0E0C0F00219B55016E9B4
:10195700F8D083D082D0E0F9D0E0FAD0E0FBC082A3
:10196700C0830219ACBBFE16E9F8D083D082D0E061
:0F197700F9D0E0FAD0E0FBC082C0830219BE2293
:10198600D083D082F8E4937012740193700DA3A3F0
:1019960093F8740193F5828883E473740293686004
:0619A600EFA3A3A380DF04
:0919AC00EBF608EAF608E9F62260
:0919B500EBF0A3EAF0A3E9F02233
:0919BE00EBF208EAF208E9F2225A
:00000001FF
